:020000020000FC
:100000000C94530AB5C2000000000000000000007C
:1000100000000000000000000000000000000000E0
:100020000000000033C00000000000005DC10000BF
:1000300000000000000000000000000000000000C0
:1000400059C1000000000000000000000000000096
:100050000000000002030406080C10182030406065
:10006000800002030406080C101820304080FF00B6
:100070000406080C10182030406080A0C0000D0D50
:100080000403060D050D0602030202004FB662FDD1
:1000900020C070FF1BC165FDFBC00994C0913701F2
:1000A000C395C0933701C5E0C519B8F3D0913701A6
:1000B000CD1B98F3C8E7089483FDC795C093B200A1
:1000C000C52DCC2329F4C0E083FDC0E8C093B20065
:1000D00009C171FF03C02B982C982D98C52D089449
:1000E00083FDC795C093B200C09339016B7FC52DC6
:1000F000CF3F09F441C0C0913801C395C093380186
:1001000070FF35C02B982C982D984FBE18957860AD
:10011000C0914001CC2391F0C0913801CA95D09193
:100120004001CD1B58F0777FC0913801D0913F013D
:10013000CD1B08F41CC02092380119C02B982C98B4
:100140002D98C1E0CA95F1F7C0911501CA95C2FD7D
:1001500009C0C1FD05C095FF299A95FD2A9A0EC0D8
:10016000289A0CC095FF2A9A95FD299A07C02B98CA
:100170002C982D984FBE1895209239014FBE189596
:10018000A5C0552021F095FF2B9A95FD2D9A2C980E
:100190009DC0552009F02C9A95FF2D9895FD2B9820
:1001A00095C0552021F095FF2D9A95FD2B9A95FF2E
:1001B0002B9895FD2D988AC095FF2A9895FD299832
:1001C00095FF299895FD2A98C1E0CA95F1F7552029
:1001D00021F095FF2B9A95FD2D9A2C9877C095FFCD
:1001E0002A9895FD29982898C1E0CA95F1F75520DD
:1001F00021F095FF2B9A95FD2D9A2C9867C0289891
:1002000095FF2A9895FD2998C1E0CA95F1F75520E8
:1002100009F02C9A95FF2D9895FD2B9857C028989A
:1002200095FF299895FD2A98C1E0CA95F1F75520C8
:1002300009F02C9A95FF2D9895FD2B9847C095FFB6
:10024000299895FD2A982898C1E0CA95F1F755207C
:1002500021F095FF2D9A95FD2B9A95FF2B9895FDF2
:100260002D9834C095FF299895FD2A9895FF2A98D6
:1002700095FD2998C1E0CA95F1F7552021F095FF29
:100280002D9A95FD2B9A95FF2B9895FD2D981EC0C4
:1002900082FF1CC0C0911501C2FD0BC0C1FD11C081
:1002A00095FF2A9895FD299895FF299895FD2A98FC
:1002B0000DC0C1FDF5CF95FF2A9895FD2998289886
:1002C00005C0289895FF299895FD2A98C52DC095B9
:1002D000089483FDC795C093B200C0933901209262
:1002E000370164604FBE18954FB6C2E0C6BB6E7F43
:1002F0004FBE18953FB68F7EADB3A170A21180613D
:10030000A0E0ADBBA0916E00AE7FA0936E0078948C
:10031000A0910601AA2349F0A92FAF7159F1A0912C
:100320000601AA95A093060125C040E050E0A9B1BE
:1003300096FDA095A2FD4FEF96FFA3E096FDA2E0EB
:10034000A0936900AA27A160ACBB8D7FA9B196FDDF
:10035000A095A2FD5FEF451741F7A0E461FDA093D2
:100360000601A92FAF7119F0A0E4A09306014093F4
:100370002D018160A0910701AA2331F0A09107010E
:10038000AA95A093070107C0A92FAF7121F0806142
:10039000AA27A160ACBB80FF30C0A0912D014A2FDD
:1003A0008E7FA92FAF7109F000C04093010171FF4A
:1003B00008C0A091010150913201A51710F050938F
:1003C000010140914E014430C1F4A09101014091DE
:1003D0000301A41B70F040916F01A40B50F0A09199
:1003E0000301A40FA093030140F4AFEFA093030116
:1003F00004C0A0910101A0930301A52DA03408F031
:100400006860A0910001A395A093000161F0F894A9
:10041000A0916E00A160A0936E0084FF02C0A1E0D5
:10042000ADBB3FBE189542E050910601552331F017
:10043000A92FAF7119F45A9550930601A0912D017F
:10044000A13018F0209230010DC02092310120928D
:100450003A01A0913001AF5FA093300118F0AFEFE7
:10046000A0933001B090010150914E01523049F4F7
:1004700066FF91F0A2E3BA1678F0A0911F01A09355
:100480000101533049F466FF39F0A2E3BA1620F0B7
:10049000A0915A01A0930101509102015B1521F036
:1004A00010F05A9501C05395509302014A95D1F628
:1004B00050913A01539509F45A9550933A01A091FD
:1004C0003B01AA95A0933B0109F046C0A1E0A0938F
:1004D0003B0145E0A0913C015A17F0F1A0913D018C
:1004E0005A1728F441E0A3E0A0933B0107C0A09174
:1004F0003E015A1718F441E040933B01D09033017C
:10050000C0900301DC14A8F0A0914E01A430D9F0F2
:1005100066FD0FC0C0923301539519F0A0913C01C4
:10052000A0933A01A1E0A0933B01ACE3A0930201A8
:1005300013C0A0913301A40F20F45FEF5093330157
:1005400002C0A0933301A0913301AF3F29F4AFEF74
:10055000A0933101A0933A01F894A0916E00A1609C
:10056000A0936E0084FF02C0A1E0ADBB3FBE189512
:100570003FB640918400509185008F7EADB3A1704D
:10058000A2118061A0E0ADBBA0916E00AE7FA093F0
:100590006E00789481FD28C096FFA2E096FDA3E04E
:1005A000A09369008260A9B196FDA095A2FF05C045
:1005B000409304015093050100C196FFA3E096FD0E
:1005C000A2E0A0936900AA27A160ACBB8D7FA92FF0
:1005D000AF7109F4E3C040E0A9B196FDA095A2FD7A
:1005E000DDC040932D01D0C096FFA3E096FDA2E0B0
:1005F000A09369008D7F61FF6CC096FFA2E096FD1D
:10060000A3E0A0936900AA27A160ACBB82604093DD
:10061000280150932901A09026014A19B090270182
:100620005B09BB24A2E0EA2EA22C483CA0E05A07BA
:1006300030F4A0E1BA2EE22CAAE0AA2E27C0483658
:10064000A1E05A0730F4A8E0BA2EE22CAFE0AA2EBF
:100650001DC0403DA2E05A0730F4A4E0BA2EE22CBF
:10066000AEE1AA2E13C0403AA5E05A0730F4A2E04A
:10067000BA2EE22CACE3AA2E09C04839A8E05A07EA
:1006800028F4A1E0BA2EE22CA8E7AA2EC42EA0914D
:100690002A01CA1AD52EA0912B01DA0ADD202AF4EC
:1006A000AFEFC094D094CA1ADA0A20922C01CA146F
:1006B000DE0418F4A1E0A0932C0140932A0150938A
:1006C0002B0140912801509129014093260150931C
:1006D0002701A09104014A1BA09105015A0B94FD2A
:1006E00046C093FD44C092FD40C05695479591FD8C
:1006F0003CC05695479590FD38C0D52EC42ED69453
:10070000C79461FD0CC0AC2DAC51AD2DA24008F0DA
:1007100045C0DD2021F4AC2DA85C08F43FC0A0E06A
:10072000EA2E97FD02C0E0906201AAEFEA0EF22CD9
:10073000F21CCE18DF084FB74170442319F040E097
:1007400050E015C0AFEFCA16D20418F04FEF50E0DA
:100750000EC0F0904701CF9C412D000C441F50E08B
:1007600008F012C04FEF50E00FC05695479594FF28
:1007700007C0552309F04FEFA42FA6954A0F521D2D
:100780004F3F520508F04FEF40932D01816061FF0C
:1007900005C0AFE1A095A923AB299A2FA0E4A093AF
:1007A0000601A92FAF7119F4AAE0A093060161FD1B
:1007B00004C0A92FAF7109F08F7EA0E2A0930701BA
:1007C000A92FAF7119F4AAE0A0930701F894A091A2
:1007D0006E00A160A0936E0084FF02C0A1E0ADBBDB
:1007E0003FBE189511E00AC013E008C01AE006C029
:1007F0001EE104C014E602C018EC00C005E1BB27EE
:10080000BA95F1F70A95D9F71A95C1F708952AE331
:1008100038E709C020E33CE806C02AE234EB03C015
:1008200025E238EC00C0652CB1E05B2E12E095FDAE
:100830009F7D95FF9062BB272898BA95F1F75520C8
:1008400009F02C9ABA95F1F72C98BA95F1F7289AF5
:10085000BA95F1F7552021F095FF2B9A95FD2D9A29
:10086000B0914801BA95F1F795FF2B9895FD2D9819
:10087000B7E8BA95F1F71A95D1F6022FB22FBA95CB
:10088000F1F70A95D9F73A9571F62898562C0895FC
:10089000221B39E0001F3A9509F40895221F211BFD
:1008A00018F4210F8894F6CF0894F4CF622C722CA0
:1008B000B0E08894B395221F331FE0F73795279552
:1008C0008894912E802E020B130B10F4192D082DF5
:1008D00010F4889401C00894661C771CBA9571F7CF
:1008E000172D062D0895322D11232AF43A950095DF
:1008F0001095031B130BF894029F712C002D129F6F
:10090000912C802C7894780C172D921C292DB4E012
:100910006B2E2695179507956A94D9F7332321F006
:1009200000951095031B130B089500914E010430A0
:1009300009F474C0B0912D01B95198F0B72FB67079
:1009400081F466FD2BC005E090906001B92DBA9549
:1009500021F00AE0BA9509F002E1B0911401B01B50
:10096000E0F066FF0AC0B0913501B0933301BFEFEC
:10097000B0933A01B1E0B0933B01B0910101B09363
:100980000301209217012092180120921901209250
:100990001A0120921B016F7B41C06064909060013E
:1009A000B92DBA9579F4B0910201B095BB1FBB1F68
:1009B0001B2FB7950B2FB12FB170B3951B2FB02FF5
:1009C000BE7F25C0B92DBA95BA9581F4B0910201C8
:1009D000B095BB1FBB1FBB1F1B2FB7950B2FB12F94
:1009E000B370B3951B2FB02FBC7F14C0B091020120
:1009F000B095BB1FBB1FBB1FBB1F1B2FB7950B2F7A
:100A0000B12FB770B395B3951B2FB02FB87FB054EB
:100A10000B2F12090093170110931801089566FF18
:100A200021C0109114011695009113010795B09102
:100A30001701B01B0B2FB0911801B10B1B2F28F41D
:100A40000038BFEF1B0740F009C00F37120508F44C
:100A500005C00FE710E002C000E81FEF00931C0183
:100A600010931D01089566FF39C000911C01B091DB
:100A700019010B0F10911D01B0911A011B1F20E0ED
:100A800030911D0133230AF42A95B0911B012B1FCD
:100A90001AF4203F40F00AC02F3008F407C00FEFCF
:100AA0001FEF2FE003C000E010E020EF30910301C2
:100AB000B09132013B1718F4332331F009C0B091E3
:100AC0001D01BB235AF004C0B0911D01BB2332F4B9
:100AD0000093190110931A0120931B01089566FFDA
:100AE00030C020916D0100911C01000F10911D017B
:100AF000111F0E94730411232AF40038BFEF1B0753
:100B000040F009C00F37120508F405C00FE710E0E8
:100B100002C000E81FEF002352F0B0910201B01BA9
:100B20000B2F18F0013008F00AC001E008C0009552
:100B30000F5FB09102010B0F08F001C00FEF00939F
:100B40001E01089566FF2EC020916E0100911A01CA
:100B500010911B010E94730411232AF40130BFEF8E
:100B60001B0740F009C00F3F120508F405C00FEF46
:100B700010E002C001E01FEF112352F0B0911E01FE
:100B8000B01B0B2F18F0013008F00AC000E008C0BD
:100B900000950F5FB0911E010B0F08F001C00FEF21
:100BA0000093030108950FEF677FB72FB670F1F43C
:100BB0006860B0911401B83008F0677FB0911401FB
:100BC000A9F00FEF109114010E944804F894B0911D
:100BD00010010B9F112D002D7894112309F00FEFB8
:100BE000B09135010B1710F40091350100933401D9
:100BF00008950E942C0974FFB0E074FDB0E0B06C61
:100C0000B0937C00B0917A00B068B064B0937A0081
:100C10000E94F20374FFB0E074FDB0E0B06CB093DA
:100C20007C00B0917A00B068B064B0937A00B09163
:100C30007A00B6FDFCCF0091780010917900B09158
:100C40007A00BF77B0937A000E94650927EE20935F
:100C5000430130E030934401732E7694622E669403
:100C6000620E731E262D372D0217130778F0809021
:100C70004301B7EEB80DB093430180904401B0E05A
:100C8000B81DB0934401260D371DEECF809043016F
:100C900090904401109144011695009143010795ED
:100CA00016950795B0914301B00FB0934101B091F3
:100CB0004401B11FB093420123E0169507952A9590
:100CC000E1F720914F012A9529F4209243012092C7
:100CD00044010AC02A9521F0800E911E2A95E1F761
:100CE0008092430190924401089520914F01B09168
:100CF0007A00B6FDFACF0091780010917900B0919A
:100D00007A00BF77B0937A00B0914501B395B09364
:100D10004501B83060F120924501B0916C01BB23D0
:100D200021F1112329F0B0914601BF3F61F009C0C4
:100D3000B09146010B1739F020F4BB2321F0BA958E
:100D400002C0B395E1F300913201B0934601B03097
:100D500050F400ECB03038F400E8B03020F400E497
:100D6000B03008F400E0009332017F7E0895213016
:100D700099F00F3FB3E01B0778F4B09143010B17D4
:100D8000B09144011B0740F4B0913201BB2359F0EC
:100D9000BA95B093320107C0B0913201BF3F19F04C
:100DA000B395B093320100913201B0910301B01BB1
:100DB00010F400910301B09133010B1750F0009132
:100DC0003301B0913301BF3F21F0B0913301B093B3
:100DD0003201502EB0914501B73009F47061089589
:100DE00002E3F894B09170010B9F012D000C001FDD
:100DF0007894B09132010B1710F0009132010093FA
:100E0000010100930301502E0093350108952092B3
:100E10001301B8E0B093140108952091200130919E
:100E20002101F8940091840010918500200F311F5A
:100E300030938900209388006160B2E0B6BB78945B
:100E400020911101309112010093110110931201B0
:100E5000021B130B2091130130911401622E732E8B
:100E6000B4E08B2EB2E09B2EB0911401B43010F0A0
:100E70008A949A94B83010F08A949A9476946794ED
:100E80008A94E1F726193709992021F016950795DC
:100E90009A94E1F7200F311F20931301309314012E
:100EA00008F00895BFEFB0931301B09314010895B3
:100EB0002091220130912301F89400918400109137
:100EC0008500020F131F1093890000938800616052
:100ED000B2E0B6BB7894089560FDFECF0E9458073B
:100EE0000895B0915E0100910E01023808F0B395AB
:100EF000003A08F0B395B63008F0B5E09B2EBCE0A0
:100F00008B2EB0911401B33030F48394839482FF1C
:100F100002C083948394B23030F48394839482FF2C
:100F200002C08394839471FF03C0B3E09B2E822C94
:100F3000109114010091130124E0169507952A954C
:100F4000E1F70819120928F0B02FB250B12FB209F9
:100F500010F402E010E0312F202F712E602E7694D5
:100F60006794B92DB330E9F0B0FD05C0060D171D2B
:100F7000262D372D06C0000F111F0250120922E046
:100F800030E0B92DB33068F020932401309325016F
:100F9000009320011093210160922201709223019D
:100FA000089500932401109325012093200130938C
:100FB00021016092220170922301089560FDFECF0D
:100FC00020912201220F30912301331FB72FB670D9
:100FD00021F02091130130911401F89400918400C4
:100FE00010918500020F131F109389000093880051
:100FF0006160B2E0B6BB78940895606120921601FA
:1010000020E004C060612092160120E2B72FB67084
:1010100009F06F7E789460FD05C0B0911601BB2386
:1010200009F0089501E063FF0AC0B0911401B330E4
:1010300008F002E0B0911401B63008F003E071FF4F
:1010400001C006E060FD06C0B0911601BB2311F09F
:10105000789408951AE083FF1AE078940000000065
:10106000F89462FD03C014E183FF14E171FF01C035
:1010700018E7B091B20030913901B31BB10B10F3F6
:10108000B0911601B395B0931601B5E03B2F6B2ECE
:10109000722CB0B7B072B21709F073943A95C9F7D1
:1010A00073947614A8F464FFB1CF6F7E30918400FE
:1010B000609085007090130180901401370D681CBA
:1010C00060928900309388006160B2E0B6BB9ECF29
:1010D00064FD9CCF0A9509F0B5CF7894089571FF0F
:1010E0000AC0B0910D01B395B0930D0160FD0CC025
:1010F00020920D0109C060FD07C064FD05C067FDB9
:1011000003C0BF91BF9122C5089520912401309161
:101110002501F8940091840010918500020F131F9F
:1011200010938900009388006160B2E0B6BB7894A8
:1011300008950E94850800E063FF03C064FF01C0BA
:1011400001E0F89410910E01B7E01B9F212D102DA6
:101150007894200F2695179526951795269517951F
:1011600010930E01183718F4B8E7B0930E010091F0
:101170000E01B0910F010B1720F060622B982C9894
:101180002D9860FDFECF0895F8942A982898299804
:1011900082FF07C0EFE1F1E073FF03C0B1E4BA954D
:1011A000F1F795FF2A9A95FD299AB2E0B0931501BF
:1011B00089C0F89495FF2D9895FD2B9882FF0DC05E
:1011C000EFE0F1E073FF0BC0289895FF299895FD9B
:1011D0002A98B1E4BA95F1F702C0E9ECF0E062FFB9
:1011E00003C0552009F02C9AB3E0B09315016AC0F2
:1011F000F8942A982898299882FF07C0EFEFF0E02A
:1012000073FF03C0B1E4BA95F1F795FF299A95FDF4
:101210002A9AB4E0B093150155C0F8942C9882FF37
:101220000DC0EFEEF0E073FF0BC095FF2A9895FD1F
:1012300029982898B1E4BA95F1F702C0E1ECF0E002
:1012400062FF06C0552021F095FF2B9A95FD2D9A3F
:10125000B5E0B093150136C0F8942A9828982998DB
:1012600082FF07C0ECEDF0E073FF03C0B1E4BA9574
:10127000F1F7289AB6E0B093150124C0F89495FFD1
:101280002B9895FD2D9882FF10C0E2E3F1E073FFEB
:101290000EC095FF2A9895FD299895FF299895FDF0
:1012A0002A98B1E4BA95F1F702C0E1EDF0E062FFEF
:1012B00006C0552021F095FF2D9A95FD2B9AB1E09F
:1012C000B09315016F7D7894089520EC30E0F9011A
:1012D0002B982C982D982A98289829986B7F0895F8
:1012E000ACE4B1E007E00D9307E00D9301E00D934E
:1012F00004E00D930FEF0D930D930BE00D9302E0BF
:101300000D9301E00D9301E00D93A8E5B1E001E03C
:101310000D9300E00D9304EB0D930FEF0D930D93E0
:101320000D9303E00D9301E00D9301E00D930FEF9A
:101330000D9305E20D9300ED0D9308E70D9308EC76
:101340000D9304E00D930DE00D9301E00D9300E08B
:101350000D930AE70D9307E00D9301E00D930895B7
:1013600020915F0109E011E0223011F405E011E065
:10137000233011F405E012E0243011F405E013E00D
:10138000253011F409E017E0263011F400E010E0F8
:1013900000933F0110934001209153018B7F777F91
:1013A000B09154019F7DB1FD90629F7BB09155013A
:1013B000B1FD9064B22FB23011F0886001C0877F18
:1013C0000895E4E5F0E000914C010A95E00FF21D6C
:1013D000B491B0936D0100914D010A95E00FF21D9B
:1013E000B491B0936E010E9465090895E2E6F0E0C1
:1013F000009167010A95E00FF21DB491B0936F015F
:101400000E9465090895E0E7F0E0009152010A9515
:10141000E00FF21DB491B09370010E946509089528
:1014200000916B01002309F40395013108F001E1FB
:10143000B02FB00FB00FB0933C011B2FB10FB10F05
:10144000B00FB0933D01B10FB00FB00FB0933E019C
:101450000895B09168010FEF1CE0B23011F400EA7A
:101460001AE0B33011F402E815E000930F01109375
:10147000100108950895209162013091630197FF52
:1014800002C020E03FEFB32FB21B6B2EB25810F416
:10149000B2E86B2E00E00395609EB12DB058D8F3F2
:1014A000009347010895F894E3E0F0E0B9E0B7BF96
:1014B000B491B078C1F3F894A895B4B7B070B4BF44
:1014C000B0916000B861B0936000B0E0B09360008C
:1014D000B4E0BEBFBFEFBDBF0E946509B0E0B5B9C3
:1014E000BFE3B4B9B0E0B8B9B0E0B7B9B0E0BBB9E8
:1014F000B0E0BAB92224A0E0B0E02D92AA31E9F719
:10150000A0E0B1E00FEF2D920A95E9F70E94700973
:101510000E94CF0D0E94B0090E94E1090E94F609C5
:101520000E94030A0E94100A0E94290A0E943A0A95
:101530000E943B0A00916401009348010E946509E2
:10154000B2E0B5BDB2E0B0938100B2E0B093B100BB
:10155000F8940E94FC030E9407040E94F8030E9472
:101560000A040E94F8030E940D040E94F8030E94DE
:10157000740E0E94FC030E94FC030E94FA03B1E077
:10158000B5BBB0936E00B2E0B6BBB0936F00B1E0F4
:10159000B7BBB0937000B0917B00B064B0937B0098
:1015A000B0917A00B460B0937A000E94F20378940C
:1015B0000E94F905B1E0BDBBBB27B160BCBB8D7F0C
:1015C0000E94FC03B1E0B0930901626025E0B09194
:1015D0002C01BB2309F425E00E94F403B0912D01F6
:1015E000B230A0F3B92FBF7100912F0100932E01EB
:1015F000B0932F01B01751F72A9549F76D7F96FFE9
:10160000B3E096FDB2E0B0936900BB27B160BCBB0C
:101610008D7F0E94FA030E94F40302E0B92FBF718C
:1016200009F400E0B0912D01B017A8F3F8940E94DE
:1016300007040E9407040E94070478940E94FC0398
:1016400020921F010E94F403B0915801B13008F4B8
:1016500086C0B0910901B13008F481C0B92FBF71C3
:10166000F1F0B0912D01BF3F08F479C0F8940E94C9
:10167000100478940E94FA03B0912D01B130B0F7B4
:10168000F8940E9407040E94F6030E9407047894CD
:101690000E94FA03B0912D01BF3F90F37AC3B8E0E6
:1016A0009B2E9068F8940E943B0A78940E94FA035B
:1016B000F8949F770E943B0A80902D01B0912D01F4
:1016C000BF37789408F453C00E94F203F8940E9444
:1016D000100478949A9429F7B82DB550B09363010B
:1016E0000E94FC03F8940E94020E0E947A0E7894E5
:1016F000BAE09B2E9068F8940E943B0A78940E946E
:10170000FA03F8949F770E943B0A80902D01B091D4
:101710002D01BF37789460F70E94F203F8940E947D
:1017200007040E94F6030E94070478949A9411F724
:10173000B82DBB5FB09362010E94FC03F8940E9435
:10174000020E0E94970E78940E94FA03F8940E9469
:101750003B0A7894B0912D01BF3FB0F31AC30091BA
:101760002D01B0911F010B1710F000931F010E9473
:10177000FA0301E0B0915401B35009F405E0B091CF
:101780002D01B01708F05ECFF8940E9410040E945B
:1017900010040E94100478940E94FC032092090116
:1017A00020920A0120920B01B0910A01B395B093E7
:1017B0000A01BF3F79F5B0910B01B395B0930B01CE
:1017C000B091660109E1BA9559F002E3BA9541F08A
:1017D0000DE7BA9529F00AEFBA9511F020920B01A6
:1017E000B0910B01B017B0F0B0910B01BA95B09366
:1017F0000B01B4EBB0930A01B0916501B0934801BD
:10180000F8940E9410047894B0916401B093480158
:101810000E94FA030E94F603B0910601BB2321F453
:10182000B92FBF7109F4D1CEB0912D01B63008F4B3
:10183000BBCF0E94FA03B0910601BB2309F4C5CEC9
:10184000F8940E94650920920101209202012092E1
:101850000301522C7894B0915101B093360120923B
:101860001701209218012092190120921A0120924A
:101870001B012092450160E070E020920E010E9461
:101880000707B8E0B093450170610E94F20374FF4E
:10189000B0E074FDB0E0B06CB0937C00B0917A0021
:1018A000B068B064B0937A00B0917A00B6FDFCCF16
:1018B0000091780010917900B0917A00BF77B093D1
:1018C0007A00112309F00FEF009346010E9475067C
:1018D000B8E0B0934501706180905301B2E0B093DD
:1018E00053010E94B00980925301F894BFEFB09366
:1018F00032010E94F006B0910101B0933201B09321
:101900003301B09334017894B1E0B0930101B09306
:1019100003015B2EB0933B01B0913101B0933A01CA
:101920007160726020920D010E942C090E943E0994
:101930000E940D070E9407070E94710705C00E94C0
:10194000B009209245017F7E95FFB5E095FDB3E09B
:10195000B06CB0937C000E9402080E946F080E9445
:1019600085080E9495040E9499080E94C4080E945C
:101970000D070E946C070E9471070E94DE07B4E009
:10198000B06CB0937C000E94FD070E946F080E941B
:1019900085080E940F050E94D3050E9499080E94A5
:1019A000D9080E940D070E946C070E9471070E94CF
:1019B000DE0795FFB3E095FDB5E0B06CB0937C0019
:1019C0000E9402080E946F080E9485080E94330549
:1019D0000E9499080E94F8080E940D070E946C0757
:1019E0000E9471070E94DE0795FFB5E095FDB3E008
:1019F000B06CB0937C000E94FD070E946F080E94AB
:101A000085080E946F050E9499080E940D090E9496
:101A10000D070E946C070E9471070E94DE07B4E068
:101A2000B06CB0937C000E9402080E946F080E9474
:101A300085080E94A2050E9499080E942C090E9414
:101A40000D070E946C070E9471070E94DE0795FF38
:101A5000B3E095FDB5E0B06CB0937C000E94FD074B
:101A600074FFB0E074FDB0E0B06CB0937C00B09156
:101A70007A00B068B064B0937A000E946F080E9448
:101A800085080E9499080E943E090E940D070E9445
:101A90006C070E9471070E9475060E94DE0771FFA5
:101AA00020C067FD1EC0B0913501B0933201B093E4
:101AB0003301B0913101B0933A01B1E0B0933B01F1
:101AC00014E624E1B0910D01B11728F07D7F746018
:101AD00020930C0106C0B0912D01B13008F034CF35
:101AE00035C072FF10C067FD0EC0B0910C01BA95F1
:101AF00011F47B7F24CFB0930C01B0912D01B13054
:101B000008F022CF23C0B0913001B13058F0B0912D
:101B10003501B0933301B0913101B0933A01B1E096
:101B2000B0933B01B0913001BA3F80F4B92FBF713F
:101B300021F4B0910601BB2349F0B091140100EFEC
:101B400067FF01C000E6B01708F4FECEF8940E94CB
:101B5000650980905301B2E0B09353010E94B0092F
:101B600080925301209201012092020120920301F0
:101B7000522C209236017E7F78940E94F2030E94BC
:101B80006509B92FBF7129F4B0910601BB2309F48F
:101B90001CCDB0915901B13008F03DCD01CEEDE042
:101BA000F0E00E94FB0D053A09F01EC0EEE0F0E007
:101BB0000E94FB0D0A3509F017C03AE0ACE4B1E031
:101BC000E3E0F0E00E94FB0D0D9331963A95D1F7DA
:101BD00035E1A8E5B1E0EFE0F0E00E94FB0D0D93E8
:101BE00031963A95D1F704C00E9470090E94020E06
:101BF000E4E2F0E00895F999FECFE1BDF2BDF89A74
:101C000000B508950E94250E3AE0ACE4B1E0E3E0AF
:101C1000F0E00D910E941D0E31963A95D1F735E115
:101C2000A8E5B1E0EFE0F0E00D910E941D0E3196C5
:101C30003A95D1F70E94300E0895F999FECF00BD74
:101C4000E1BDF2BDFA9AF99A0895EDE0F0E00FEFE8
:101C50000E941D0EEEE0F0E00FEF0E941D0E0895B1
:101C6000EDE0F0E005EA0E941D0EEEE0F0E00AE58E
:101C70000E941D0E08953091490100914A013130B2
:101C800011F400934C01323011F400934D013330C4
:101C900011F400934E01343011F40093600135309B
:101CA00011F400934F01363011F400935201373094
:101CB00011F400935E01383011F40093670139305C
:101CC00011F400935F013A3011F4009353013B305B
:101CD00011F4009368013C3011F4009354013D303D
:101CE00011F400935501089525E00E94FC032A9504
:101CF000E1F708950E9407040E940A040E940D045F
:101D00000E9410040E94F6030E9407040E940A0425
:101D10000E940D040E9410040E94F6030E94070412
:101D20000E940A040E940D040E94100408950E945B
:101D300010040E940D040E940A040E9407040E94DD
:101D4000F6030E9410040E940D040E940A040E94DF
:101D500007040E94F6030E9410040E940D040E94D2
:101D60000A040E94070408958090490190904A0156
:101D70000E9407040E9407040E9407040E94F603C1
:101D80008A94B1F70E9410040E94F6039A94D1F746
:101D90000895F8940E947A0E78940E94740E0E941E
:101DA000740EB1E0B0934901B1E0B0934A012092C2
:101DB0004B01F8940E94B40E7894B5E06B2E7090AD
:101DC0002D010E94FC03B0912D017B16C1F7B130AB
:101DD00018F0BF3F70F10CC00E943B0EF8940E94B7
:101DE000020E0E947A0EB8E0B09360000E94740E5A
:101DF0006A9429F7B0914B01B395B0934B01B3307E
:101E000008F4D7CF0E94740EB0914A01B395B093F5
:101E10004A01F894B0914901BA95EEE7F0E0EB0F72
:101E2000F21D049178940395B0914A01B01708F41B
:101E3000BECF0E94740E0E94740EB0914901B395FA
:101E4000B0934901B0914901BE3008F4ADCF0E9472
:101E50007009F8940E94020EB8E0B09360000E94EE
:021E6000740EFE
:00000001FF
